:020000040000FA
:0408000063EF09F0A9
:1008100003B283EF05F0F2B4A1EF05F09EB0A9EFAB
:1008200005F09EB2B1EF05F0F2A81AEF04F0F2B2B3
:1008300032EF04F09EB61FEF04F012EF09F09E961F
:1008400000011450000A06E000011450010A06E0FD
:1008500012EF09F075EC20F012EF09F06DEC22F0C8
:1008600012EF09F0CD90F2929EA03CEF04F001014E
:10087000533F3CEF04F0542BAEC1B2F1AFC1B3F122
:10088000B0C1B4F1B1C1B5F1AAC1AEF1ABC1AFF124
:10089000ACC1B0F1ADC1B1F1A6C1AAF1A7C1ABF134
:1008A000A8C1ACF1A9C1ADF1A2C1A6F1A3C1A7F144
:1008B000A4C1A8F1A5C1A9F19EC1A2F19FC1A3F154
:1008C000A0C1A4F1A1C1A5F19AC19EF19BC19FF164
:1008D0009CC1A0F19DC1A1F196C19AF197C19BF174
:1008E00098C19CF199C19DF1CECF96F1CFCF97F1F0
:1008F00053C198F154C199F1CF6ACE6A0101536B8B
:10090000546B9E90CD800FBC0F8E0FBA8BEF04F00E
:100910000F8A12EF09F00F8C0FBEC7EF04F096C1DB
:100920009AF197C19BF198C19CF199C19DF19AC12F
:100930009EF19BC19FF19CC1A0F19DC1A1F19EC1FF
:10094000A2F19FC1A3F1A0C1A4F1A1C1A5F1A2C1CF
:10095000A6F1A3C1A7F1A4C1A8F1A5C1A9F1A6C19F
:10096000AAF1A7C1ABF1A8C1ACF1A9C1ADF1AAC16F
:10097000AEF1ABC1AFF1ACC1B0F1ADC1B1F1AEC13F
:10098000B2F1AFC1B3F1B0C1B4F1B1C1B5F1010180
:100990005E6B5F6B606B616B96515E2797515F2357
:1009A00098516023995161239A515E279B515F238F
:1009B0009C5160239D5161239E515E279F515F236F
:1009C000A0516023A1516123A2515E27A3515F234F
:1009D000A4516023A5516123A6515E27A7515F232F
:1009E000A8516023A9516123AA515E27AB515F230F
:1009F000AC516023AD516123AE515E27AF515F23EF
:100A0000B0516023B1516123B2515E27B3515F23CE
:100A1000B4516023B5516123D89001016133603333
:100A20005F335E33D8900101613360335F335E33EF
:100A3000D8900101613360335F335E3300C10CF144
:100A400001C10DF102C10EF103C10FF104C110F19A
:100A500005C111F106C112F107C113F108C114F16A
:100A600009C115F10AC116F10BC117F134C135F1F5
:100A700011B846EF05F00101620E046F010E056F1B
:100A8000000E066F000E076F4FEF05F00101A70E75
:100A9000046F020E056F000E066F000E076F5EC139
:100AA00000F15FC101F160C102F161C103F10CEC21
:100AB0001FF003BF04D019BE02D019A0108C11A0E2
:100AC00067EF05F010BA67EF05F00F80108A0CC1D0
:100AD00000F10DC101F10EC102F10FC103F110C10E
:100AE00004F111C105F112C106F113C107F114C1DE
:100AF00008F115C109F116C10AF117C10BF135C191
:100B000034F112EF09F00392ABB2AB98AB8803015A
:100B100003EE00F080517F0BE92604C0EFFF802B2D
:100B20008151805D700BD8A48B8200008051815D63
:100B3000700BD8A48B9281518019D8B4079012EF12
:100B400009F0F2940101453F12EF09F0462B12EF34
:100B500009F09E900101533F12EF09F0542B12EF60
:100B600009F09E9211B820EF07F08BB4BFEF05F0AB
:100B700010ACBFEF05F08B84109CC0EF05F08B9498
:100B8000C3CF55F1C4CF56F1C28207B42AEF06F0A5
:100B900047C14BF148C14CF149C14DF14AC14EF139
:100BA0005EC162F15FC163F160C164F161C165F171
:100BB00096C1B6F197C1B7F198C1B8F199C1B9F131
:100BC0009AC1BAF19BC1BBF19CC1BCF19DC1BDF101
:100BD0009EC1BEF19FC1BFF1A0C1C0F1A1C1C1F1D1
:100BE000A2C1C2F1A3C1C3F1A4C1C4F1A5C1C5F1A1
:100BF000A6C1C6F1A7C1C7F1A8C1C8F1A9C1C9F171
:100C0000AAC1CAF1ABC1CBF1ACC1CCF1ADC1CDF140
:100C1000AEC1CEF1AFC1CFF1B0C1D0F1B1C1D1F110
:100C2000B2C1D2F1B3C1D3F1B4C1D4F1B5C1D5F1E0
:100C3000010155515B2756515C23E86A5D230E2E56
:100C40002AEF06F05CC157F15DC158F15B6B5C6B3C
:100C50005D6B078E0201002F12EF09F03C0E006F52
:100C60001A50E00BE00AE866128818BE02D018B4E9
:100C7000108E00C10CF101C10DF102C10EF103C1D2
:100C80000FF104C110F105C111F106C112F107C144
:100C900013F108C114F109C115F10AC116F10BC114
:100CA00017F134C135F101018A675EEF06F08B67F9
:100CB0005EEF06F08C675EEF06F08D6762EF06F080
:100CC00092EF06F08EC100F18FC101F190C102F1E7
:100CD00091C103F10101010E046F000E056F000EBA
:100CE000066F000E076F0CEC1FF000C18EF101C102
:100CF0008FF102C190F103C191F1006787EF06F017
:100D0000016787EF06F0026787EF06F0036792EF4F
:100D100006F08AC18EF18BC18FF18CC190F18DC12B
:100D200091F10F80D57ED5BE6DD0D6CF47F1D7CF0C
:100D300048F145C149F1E86AE8CF4AF119BE02D04D
:100D400019A0108C109047C100F148C101F149C1B0
:100D500002F14AC103F101010A0E046F000E056F92
:100D6000000E066F000E076F0CEC1FF003AF108033
:100D7000010154A7C8EF06F00F9A0F9C0F9E0101C6
:100D8000000E5E6F600E5F6F3D0E606F080E616F4C
:100D9000010147BFD8EF06F04867D8EF06F0496772
:100DA000D8EF06F04A67D8EF06F0F288FDEF06F0BC
:100DB000F2985E6B5F6B606B616B966B976B986B79
:100DC000996B9A6B9B6B9C6B9D6B9E6B9F6BA06BE7
:100DD000A16BA26BA36BA46BA56BA66BA76BA86B97
:100DE000A96BAA6BAB6BAC6BAD6BAE6BAF6BB06B47
:100DF000B16BB26BB36BB46BB56BD76AD66A0101DA
:100E0000456B466B0CC100F10DC101F10EC102F141
:100E10000FC103F110C104F111C105F112C106F1B6
:100E200013C107F114C108F115C109F116C10AF186
:100E300017C10BF135C134F112EF09F012EF09F0CF
:100E40000201002F79EF08F0D59ED6CF47F1D7CF1A
:100E500048F145C149F1E86AE8CF4AF1D76AD66A54
:100E60000101456B466BD58E1A50E00BE00AE8662F
:100E7000128818BE02D018B4108E17AE1C8C00C198
:100E80000CF101C10DF102C10EF103C10FF104C15A
:100E900010F105C111F106C112F107C113F108C12A
:100EA00014F109C115F10AC116F10BC117F134C1D2
:100EB00035F10FA0109A11B869EF07F00101620E29
:100EC000046F010E056F000E066F000E076F72EFC4
:100ED00007F00101A70E046F020E056F000E066FEA
:100EE000000E076F47C100F148C101F149C102F18D
:100EF0004AC103F10CEC1FF003BF85EF07F019BEE8
:100F000002D019A0108C11B00F800CC100F10DC1DE
:100F100001F10EC102F10FC103F110C104F111C1C1
:100F200005F112C106F113C107F114C108F115C191
:100F300009F116C10AF117C10BF135C134F10201F3
:100F40003C0E006F00C10CF101C10DF102C10EF1A8
:100F500003C10FF104C110F105C111F106C112F175
:100F600007C113F108C114F109C115F10AC116F145
:100F70000BC117F134C135F101018A67C7EF07F0E2
:100F80008B67C7EF07F08C67C7EF07F08D67CBEF74
:100F900007F0FBEF07F08EC100F18FC101F190C1A6
:100FA00002F191C103F10101010E046F000E056F02
:100FB000000E066F000E076F0CEC1FF000C18EF1E3
:100FC00001C18FF102C190F103C191F10067F0EF0F
:100FD00007F00167F0EF07F00267F0EF07F0036733
:100FE000FBEF07F08AC18EF18BC18FF18CC190F1BC
:100FF0008DC191F10F80109047C100F148C101F1FE
:1010000049C102F14AC103F101010A0E046F000E49
:10101000056F000E066F000E076F0CEC1FF003AF9C
:101020001080010154A721EF08F00F9A0F9C0F9E2A
:101030000101000E5E6F600E5F6F3D0E606F080E67
:10104000616F47C100F148C101F149C102F14AC1D4
:1010500003F10101140E046F050E056F000E066FFB
:10106000000E076F0CEC1FF003AF3AEF08F0F288A8
:101070005FEF08F0F2985E6B5F6B606B616B966B75
:10108000976B986B996B9A6B9B6B9C6B9D6B9E6B34
:101090009F6BA06BA16BA26BA36BA46BA56BA66BE4
:1010A000A76BA86BA96BAA6BAB6BAC6BAD6BAE6B94
:1010B000AF6BB06BB16BB26BB36BB46BB56B0CC198
:1010C00000F10DC101F10EC102F10FC103F110C118
:1010D00004F111C105F112C106F113C107F114C1E8
:1010E00008F115C109F116C10AF117C10BF135C19B
:1010F00034F12CEC23F01D661ED01CAE11D01C9ECA
:101100001D8E18AE07D0146A040E156E166A75ECA3
:1011100020F011D0146A156A166A75EC20F00BD015
:101120001CAC09D01C9C1D8C010E146E156A166A2D
:101130006DEC22F000D08BB4A5EF08F010ACA5EF59
:1011400008F08B84109CA6EF08F08B94C3CF55F168
:10115000C4CF56F1C28207B410EF09F047C14BF17A
:1011600048C14CF149C14DF14AC14EF15EC162F135
:101170005FC163F160C164F161C165F196C1B6F10F
:1011800097C1B7F198C1B8F199C1B9F19AC1BAF153
:101190009BC1BBF19CC1BCF19DC1BDF19EC1BEF123
:1011A0009FC1BFF1A0C1C0F1A1C1C1F1A2C1C2F1F3
:1011B000A3C1C3F1A4C1C4F1A5C1C5F1A6C1C6F1C3
:1011C000A7C1C7F1A8C1C8F1A9C1C9F1AAC1CAF193
:1011D000ABC1CBF1ACC1CCF1ADC1CDF1AEC1CEF163
:1011E000AFC1CFF1B0C1D0F1B1C1D1F1B2C1D2F133
:1011F000B3C1D3F1B4C1D4F1B5C1D5F10101555199
:101200005B2756515C23E86A5D230E2E10EF09F030
:101210005CC157F15DC158F15B6B5C6B5D6B078E18
:1012200012EF09F002C0E0FF005001C0D8FF10002B
:10123000A6B218EF09F00CC0A9FF0BC0A8FFA69E2C
:10124000A69CA684F29E550EA76EAA0EA76EA68235
:10125000F28EA694A6B22AEF09F00C2A1200A96E0B
:10126000A69EA69CA680A8500C2A120004012C0E53
:10127000826F3BEC0BF007EC20F00C502FEC09F0E8
:10128000E8CF00F10C502FEC09F0E8CF01F101AFED
:101290004FEF09F00101FF0E026FFF0E036FAAEC82
:1012A0001FF029675BEF09F00401200E826F3BEC11
:1012B0000BF060EF09F004012D0E826F3BEC0BF098
:1012C000B4EC1DF01200306A076A0F6A106A116AE6
:1012D000126A136A0F010E0EC16E860EC06E030EE7
:1012E000C26E0F01896A110E926E080E8A6EF10E9F
:1012F000936E8B6A980E946EF18EFC0E2FEC09F0B3
:10130000E8CF0BF00BA011800BA211820BA411846B
:101310000BA81188C90E2FEC09F0E8CF17F0CA0E00
:101320002FEC09F0E8CF18F0CB0E2FEC09F0E8CF46
:1013300019F0CC0E2FEC09F0E8CF1AF0CD0E2FECFF
:1013400009F0E8CF2FF01C6A1D6A0E6A01015B6B81
:101350005C6B5D6B576B586BF29A0101476B486B86
:10136000496B4A6B4B6B4C6B4D6B4E6B4F6B506BC1
:10137000516B526B456B466BD76AD66A0F01280ECC
:10138000D56EF28A9D90B00ECD6E01015E6B5F6BE3
:10139000606B616B626B636B646B656B666B676BD9
:1013A000686B696B536B546BCF6ACE6A0F9A0F9C54
:1013B0000F9E9D80760ECA6E9D8202013C0E006FCC
:1013C000CC6A160E2FEC09F0E8CF00F1170E2FECC7
:1013D00009F0E8CF01F1180E2FEC09F0E8CF02F187
:1013E000190E2FEC09F0E8CF03F1010103AF13EF61
:1013F0000AF007EC20F0160E0C6E00C10BF018EC92
:1014000009F0170E0C6E01C10BF018EC09F0180E64
:101410000C6E02C10BF018EC09F0190E0C6E03C132
:101420000BF018EC09F000C18AF101C18BF102C187
:101430008CF103C18DF100C18EF101C18FF102C1A8
:1014400090F103C191F11A0E2FEC09F0E8CF00F1F1
:101450001B0E2FEC09F0E8CF01F11C0E2FEC09F068
:10146000E8CF02F11D0E2FEC09F0E8CF03F10101E6
:1014700003AF69EF0AF007EC20F01A0E0C6E00C102
:101480000BF018EC09F01B0E0C6E01C10BF018EC00
:1014900009F01C0E0C6E02C10BF018EC09F01D0EC9
:1014A0000C6E03C10BF018EC09F01A0E2FEC09F0CA
:1014B000E8CF00F11B0E2FEC09F0E8CF01F11C0E74
:1014C0002FEC09F0E8CF02F11D0E2FEC09F0E8CF68
:1014D00003F100C192F101C193F102C194F103C182
:1014E00095F1240EAC6E900EAB6E240EAC6E080E11
:1014F000B86E000EB06E1F0EAF6E0401806B816B74
:101500000F01900EAB6E0F019D8A0301806B816B02
:10151000C26B8B92146A156A166A9D860790000149
:10152000F28EF28C07B05DEF1CF00FB0FCEF15F0FF
:1015300010BEFCEF15F012B8FCEF15F0030180515E
:1015400081197F0BD8B45DEF1CF013EE00F08151D0
:101550007F0BE126812BE7CFE8FFE00BD8B45DEFEE
:101560001CF023EE82F0C2513F0BD926E7CFDFFFFC
:10157000C22BDF50780AD8A45DEF1CF007808EC123
:1015800000F18FC101F190C102F191C103F101019C
:10159000040E046F000E056F000E066F000E076F3D
:1015A0000CEC1FF000AFDEEF0AF00101030E8E6FAE
:1015B000000E8F6F000E906F000E916F030182512D
:1015C000720AD8B4E1EF15F08251520AD8B4E1EFB3
:1015D00015F08251750AD8B4E1EF15F08251630A13
:1015E000D8B417EF19F08251690AD8B488EF12F015
:1015F00082517A0AD8B49BEF13F08251490AD8B4C9
:1016000027EF12F08251500AD8B431EF11F0825115
:10161000700AD8B479EF11F08251540AD8B4A9EF06
:1016200011F08251740AD8B4F4EF11F08251410ADA
:10163000D8B451EF0CF082514B0AD8B44FEF0BF0F5
:1016400082516D0AD8B484EF10F082514D0AD8B49B
:101650009DEF10F08251730AD8B411EF15F082514A
:10166000530AD8B476EF15F08251590AD8B4D5EFA1
:101670000FF04EEF19F0040114EE00F080517F0BD3
:10168000E12682C4E7FF802B120004010D0E826F59
:101690003BEC0BF00A0E826F3BEC0BF012000401E6
:1016A0004B0E826F3BEC0BF004012C0E826F3BEC77
:1016B0000BF081B802D02FB630D003018351430A1A
:1016C000D8B494EF0BF003018351630AD8B496EFBA
:1016D0000BF003018351520AD8B498EF0BF00301C9
:1016E0008351720AD8B49AEF0BF003018351470A71
:1016F000D8B49CEF0BF003018351670AD8B49EEF76
:101700000BF003018351540AD8B4A0EF0BF003018E
:101710008351740AD8B40FEF0CF003018351550ABA
:10172000D8B4A2EF0BF082D02F807AD02F9078D04F
:101730002F8276D02F9274D02F8472D02F9470D0B5
:101740002F866ED084C330F185C331F186C332F168
:1017500087C333F10101296B55EC20F0CCEC1FF06D
:1017600000C104F101C105F102C106F103C107F195
:1017700048EC20F0200EF86EF76AF66A0900F5CF03
:101780002CF10900F5CF2DF10900F5CF2EF109005C
:10179000F5CF2FF10900F5CF30F10900F5CF31F188
:1017A0000900F5CF32F10900F5CF33F10101296BC2
:1017B00055EC20F0CCEC1FF00CEC1FF00067E8EFCC
:1017C0000BF00167E8EF0BF00267E8EF0BF003673F
:1017D00001D025D004014E0E826F3BEC0BF00401CA
:1017E0006F0E826F3BEC0BF004014D0E826F3BECF1
:1017F0000BF00401610E826F3BEC0BF00401740EE0
:10180000826F3BEC0BF00401630E826F3BEC0BF03C
:101810000401680E826F3BEC0BF04CEF19F02F9631
:10182000CD0E0C6E2FC00BF018EC09F0CD0E2FEC86
:1018300009F0E8CF2FF02FB006D00401630E826FBD
:101840003BEC0BF005D00401430E826F3BEC0BF038
:101850002FB206D00401720E826F3BEC0BF005D064
:101860000401520E826F3BEC0BF02FB406D0040142
:10187000670E826F3BEC0BF005D00401470E826FC0
:101880003BEC0BF02FB606D00401740E826F3BECDC
:101890000BF005D00401540E826F3BEC0BF04CEFC3
:1018A00019F00401410E826F3BEC0BF003018351F0
:1018B000310AD8B4F5EF0EF003018351320AD8B4DF
:1018C00025EF0EF003018351330AD8B4AEEF0DF0CB
:1018D00003018351340AD8B49EEF0CF00301835105
:1018E000350AD8B47BEF0CF004013F0E826F3BEC5D
:1018F0000BF04CEF19F004012C0E826F3BEC0BF057
:1019000003018451300AD8B48EEF0CF003018451E6
:10191000310AD8B496EF0CF0E7EF0DF08B9004018C
:10192000300E826F3BEC0BF09CEF0CF08B800401CF
:10193000310E826F3BEC0BF04CEF19F0CC0E2FEC1C
:1019400009F0E8CF0BF004012C0E826F3BEC0BF09A
:1019500003018451310AD8B4C2EF0CF00301845161
:10196000300AD8B4C4EF0CF0030184514D0AD8B446
:10197000CEEF0CF003018451540AD8B4D5EF0CF02B
:10198000ECEF0CF08A8401D08A940BAE04D00BAC3F
:1019900002D00BBA21D0E00E0B1218D01F0E0B167E
:1019A0008539E844E00B0B1211D0E00E0B1648EC21
:1019B00020F085C332F186C333F10101296B55EC68
:1019C00020F0CCEC1FF000511F0B0B12CC0E0C6E54
:1019D0000BC00BF018EC09F00401340E826F3BECE5
:1019E0000BF004012C0E826F3BEC0BF0CC0E2FECB5
:1019F00009F0E8CF1AF08AB406D00401300E826FE5
:101A00003BEC0BF005D00401310E826F3BEC0BF088
:101A100004012C0E826F3BEC0BF01A38E840070BE8
:101A2000E8CF82F40401300E82273BEC0BF0040176
:101A30002C0E826F3BEC0BF007EC20F01A501F0BC2
:101A4000E8CF00F1AAEC1FF032C182F40401300E9D
:101A500082273BEC0BF033C182F40401300E822765
:101A60003BEC0BF004012C0E826F3BEC0BF007EC0F
:101A700020F02DC000F100AF0BD0FF0E016FFF0E64
:101A8000026FFF0E036F04012D0E826F3BEC0BF013
:101A9000AAEC1FF031C182F40401300E82273BEC26
:101AA0000BF032C182F40401300E82273BEC0BF0C4
:101AB00033C182F40401300E82273BEC0BF00401A9
:101AC0002C0E826F3BEC0BF007EC20F02CC000F1E9
:101AD000AAEC1FF031C182F40401300E82273BECE6
:101AE0000BF032C182F40401300E82273BEC0BF084
:101AF00033C182F40401300E82273BEC0BF0040169
:101B00002C0E826F3BEC0BF007EC20F02EC000F1A6
:101B100000AF0BD0FF0E016FFF0E026FFF0E036FC1
:101B200004012D0E826F3BEC0BF0AAEC1FF031C1CB
:101B300082F40401300E82273BEC0BF032C182F4B8
:101B40000401300E82273BEC0BF033C182F4040118
:101B5000300E82273BEC0BF04CEF19F0CB0E2FEC44
:101B600009F0E8CF0BF004012C0E826F3BEC0BF078
:101B700003018451450AD8B4D2EF0DF0030184511A
:101B8000440AD8B4D5EF0DF003018451300AD8B41B
:101B9000D8EF0DF003018451310AD8B4DCEF0DF019
:101BA000E7EF0DF00B9EE1EF0DF00B8EE1EF0DF086
:101BB000FC0E0B16E1EF0DF0FC0E0B160B80E1EFA7
:101BC0000DF0CB0E0C6E0BC00BF018EC09F00401FD
:101BD000330E826F3BEC0BF004012C0E826F3BEC5A
:101BE0000BF0CB0E2FEC09F0E8CF19F019BE00EF87
:101BF0000EF00401450E826F3BEC0BF005EF0EF08A
:101C00000401440E826F3BEC0BF004012C0E826F3A
:101C10003BEC0BF00401300E826F3BEC0BF0040147
:101C20002C0E826F3BEC0BF019B01EEF0EF004018E
:101C3000300E826F3BEC0BF023EF0EF00401310EFF
:101C4000826F3BEC0BF04CEF19F0CA0E2FEC09F051
:101C5000E8CF0BF004012C0E826F3BEC0BF003017C
:101C60008451450AD8B461EF0EF003018451440A4F
:101C7000D8B464EF0EF0030184514D0AD8B46DEF6F
:101C80000EF003018451410AD8B467EF0EF003014E
:101C90008451460AD8B46AEF0EF003018451560A03
:101CA000D8B475EF0EF003018451500AD8B480EF18
:101CB0000EF003018451520AD8B483EF0EF08CEF7A
:101CC0000EF00B9E86EF0EF00B8E86EF0EF00B9C47
:101CD00086EF0EF00B8C86EF0EF0FC0E0B1685C314
:101CE000E8FF030B0B1286EF0EF0C70E0B1685C331
:101CF000E8FF070BE846E846E8460B1286EF0EF0D1
:101D00000B8486EF0EF00B9486EF0EF0CA0E0C6E6D
:101D10000BC00BF018EC09F0CA0E2FEC09F0E8CF5D
:101D200018F00401320E826F3BEC0BF004012C0E14
:101D3000826F3BEC0BF018BEA5EF0EF00401450ED0
:101D4000826F3BEC0BF0AAEF0EF00401440E826FA1
:101D50003BEC0BF004012C0E826F3BEC0BF018C037
:101D6000E8FF030BE8CF82F40401300E82273BEC3E
:101D70000BF004012C0E826F3BEC0BF018BCC8EF8B
:101D80000EF00401410E826F3BEC0BF0CDEF0EF034
:101D90000401460E826F3BEC0BF004012C0E826FA7
:101DA0003BEC0BF018C0E8FF380BE842E842E84291
:101DB000E8CF82F40401300E82273BEC0BF00401E3
:101DC0002C0E826F3BEC0BF018B4EEEF0EF004011A
:101DD000520E826F3BEC0BF0F3EF0EF00401500E4D
:101DE000826F3BEC0BF04CEF19F0C90E2FEC09F0B1
:101DF000E8CF0BF004012C0E826F3BEC0BF00301DB
:101E00008451450AD8B413EF0FF003018451440AFA
:101E1000D8B416EF0FF0030184514D0AD8B419EF6E
:101E20000FF027EF0FF00B9E21EF0FF00B8E21EF3D
:101E30000FF0F80E0B1685C3E8FF070B0B1221EF0E
:101E40000FF0C90E0C6E0BC00BF018EC09F004017A
:101E5000310E826F3BEC0BF004012C0E826F3BECD9
:101E60000BF0C90E2FEC09F0E8CF17F017BE06D023
:101E70000401450E826F3BEC0BF005D00401440ECB
:101E8000826F3BEC0BF004012C0E826F3BEC0BF0ED
:101E900017C0E8FF070BE8CF82F40401300E822759
:101EA0003BEC0BF004012C0E826F3BEC0BF0078037
:101EB00007EC20F028C0E8FF003B00430043030B81
:101EC000AAEC1FF033C182F40401300E82273BECF0
:101ED0000BF004012C0E826F3BEC0BF007EC20F0B2
:101EE00028C001F1019F019D29C000F10101AAEC68
:101EF0001FF02FC182F40401300E82273BEC0BF05F
:101F000030C182F40401300E82273BEC0BF031C16A
:101F100082F40401300E82273BEC0BF032C182F4D4
:101F20000401300E82273BEC0BF033C182F4040134
:101F3000300E82273BEC0BF004012C0E826F3BEC41
:101F40000BF007EC20F02AC001F12BC000F1D89073
:101F500001330033D890013300330101AAEC1FF0A4
:101F60002FC182F40401300E82273BEC0BF030C10C
:101F700082F40401300E82273BEC0BF031C182F475
:101F80000401300E82273BEC0BF032C182F40401D5
:101F9000300E82273BEC0BF033C182F40401300E8B
:101FA00082273BEC0BF04CEF19F0FC0E2FEC09F004
:101FB000E8CF0BF003018351520AD8B40CEF10F0B4
:101FC00003018351720AD8B40FEF10F0030183515B
:101FD000500AD8B412EF10F003018351700AD8B43C
:101FE00015EF10F003018351550AD8B418EF10F023
:101FF00003018351750AD8B41BEF10F0030183511C
:10200000430AD8B424EF10F003018351630AD8B413
:1020100027EF10F030EF10F00B902AEF10F00B804C
:102020002AEF10F00B922AEF10F00B822AEF10F03B
:102030000B942AEF10F00B842AEF10F00B962AEF86
:1020400010F00B862AEF10F00B982AEF10F00B8897
:102050002AEF10F0FC0E0C6E0BC00BF018EC09F020
:102060000401590E826F3BEC0BF011901192119408
:102070001198FC0E2FEC09F0E8CF0BF00BA01180AB
:102080000BA211820BA411840BA8118811A050EF90
:1020900010F00401520E826F3BEC0BF055EF10F084
:1020A0000401720E826F3BEC0BF011A85FEF10F091
:1020B0000401430E826F3BEC0BF064EF10F004015F
:1020C000630E826F3BEC0BF011A26EEF10F0040177
:1020D000500E826F3BEC0BF073EF10F00401700EAA
:1020E000826F3BEC0BF011A47DEF10F00401550E54
:1020F000826F3BEC0BF082EF10F00401750E826FE3
:102100003BEC0BF04CEF19F004016D0E826F3BECD1
:102110000BF003018351300AD8B4E1EF10F0030152
:102120008351310AD8B4F4EF10F003018351320A1D
:10213000D8B407EF11F04EEF19F081B803D02FB4E7
:102140004CEF19F004014D0E826F3BEC0BF048ECA4
:1021500020F084C331F185C332F186C333F101012C
:10216000296B55EC20F0CCEC1FF003018351300AB1
:10217000D8B4C9EF10F003018351310AD8B4D1EFBC
:1021800010F003018351320AD8B4D9EF10F04EEFAA
:1021900019F0FD0E0C6E00C10BF018EC09F0E1EF28
:1021A00010F0FE0E0C6E00C10BF018EC09F0F4EF0D
:1021B00010F0FF0E0C6E00C10BF018EC09F007EFE9
:1021C00011F00401300E826F3BEC0BF004012C0E79
:1021D000826F3BEC0BF007EC20F0FD0E2FEC09F0CA
:1021E000E8CF00F118EF11F00401310E826F3BECE3
:1021F0000BF004012C0E826F3BEC0BF007EC20F08F
:10220000FE0E2FEC09F0E8CF00F118EF11F00401F9
:10221000320E826F3BEC0BF007EC20F004012C0E29
:10222000826F3BEC0BF0FF0E2FEC09F0E8CF00F1D2
:10223000AAEC1FF031C182F40401300E82273BEC7E
:102240000BF032C182F40401300E82273BEC0BF01C
:1022500033C182F40401300E82273BEC0BF04CEFCB
:1022600019F081B803D02FB227EF12F083C32AF1FF
:1022700084C32BF185C32CF186C32DF187C32EF1C6
:1022800088C32FF189C330F18AC331F18BC332F196
:102290008CC333F1010155EC20F0CCEC1FF0160E8D
:1022A0000C6E00C10BF018EC09F0170E0C6E01C19A
:1022B0000BF018EC09F0180E0C6E02C10BF018ECC4
:1022C00009F0190E0C6E03C10BF018EC09F000C1F7
:1022D0008AF101C18BF102C18CF103C18DF100C102
:1022E0008EF101C18FF102C190F103C191F127EF8D
:1022F00012F081B803D02FB227EF12F083C32AF176
:1023000084C32BF185C32CF186C32DF187C32EF135
:1023100088C32FF189C330F18AC331F18BC332F105
:102320008CC333F1010155EC20F0CCEC1FF000C15F
:102330008AF101C18BF102C18CF103C18DF100C1A1
:102340008EF101C18FF102C190F103C191F127EF2C
:1023500012F081B803D02FB227EF12F083C32AF115
:1023600084C32BF185C32CF186C32DF187C32EF1D5
:1023700088C32FF189C330F18AC331F18CC332F1A4
:102380008DC333F1010155EC20F0CCEC1FF00101BD
:10239000000E046F000E056F010E066F000E076F32
:1023A0001DEC1FF01A0E0C6E00C10BF018EC09F0BA
:1023B0001B0E0C6E01C10BF018EC09F01C0E0C6E1C
:1023C00002C10BF018EC09F01D0E0C6E03C10BF0EE
:1023D00018EC09F000C192F101C193F102C194F12E
:1023E00003C195F127EF12F081B803D02FB227EF88
:1023F00012F083C32AF184C32BF185C32CF186C369
:102400002DF187C32EF188C32FF189C330F18AC320
:1024100031F18CC332F18DC333F1010155EC20F061
:10242000CCEC1FF00101000E046F000E056F010ED1
:10243000066F000E076F1DEC1FF000C192F101C185
:1024400093F102C194F103C195F127EF12F0160E3A
:102450002FEC09F0E8CF00F1170E2FEC09F0E8CFD0
:1024600001F1180E2FEC09F0E8CF02F1190E2FEC54
:1024700009F0E8CF03F1AAEC1FF06DEC1DF00401A8
:10248000730E826F3BEC0BF004012C0E826F3BEC61
:102490000BF08AC100F18BC101F18CC102F18DC139
:1024A00003F1AAEC1FF06DEC1DF00401730E826FB6
:1024B0003BEC0BF004012C0E826F3BEC0BF01A0E80
:1024C0002FEC09F0E8CF00F11B0E2FEC09F0E8CF5C
:1024D00001F11C0E2FEC09F0E8CF02F11D0E2FECDC
:1024E00009F0E8CF03F169EC19F004012C0E826FBA
:1024F0003BEC0BF092C100F193C101F194C102F1E8
:1025000095C103F169EC19F045EC0BF04EEF19F0B1
:102510000401690E826F3BEC0BF004012C0E826FFC
:102520003BEC0BF00101040E006F000E016F000E7A
:10253000026F000E036FAAEC1FF02CC182F404019D
:10254000300E82273BEC0BF02DC182F40401300EDB
:1025500082273BEC0BF02EC182F40401300E82275F
:102560003BEC0BF02FC182F40401300E82273BECD0
:102570000BF030C182F40401300E82273BEC0BF0EB
:1025800031C182F40401300E82273BEC0BF032C1E2
:1025900082F40401300E82273BEC0BF033C182F44D
:1025A0000401300E82273BEC0BF004012C0E826FED
:1025B0003BEC0BF00101030E006F000E016F000EEB
:1025C000026F000E036FAAEC1FF02CC182F404010D
:1025D000300E82273BEC0BF02DC182F40401300E4B
:1025E00082273BEC0BF02EC182F40401300E8227CF
:1025F0003BEC0BF02FC182F40401300E82273BEC40
:102600000BF030C182F40401300E82273BEC0BF05A
:1026100031C182F40401300E82273BEC0BF032C151
:1026200082F40401300E82273BEC0BF033C182F4BC
:102630000401300E82273BEC0BF004012C0E826F5C
:102640003BEC0BF00101350E006F000E016F000E28
:10265000026F000E036FAAEC1FF02CC182F404017C
:10266000300E82273BEC0BF02DC182F40401300EBA
:1026700082273BEC0BF02EC182F40401300E82273E
:102680003BEC0BF02FC182F40401300E82273BECAF
:102690000BF030C182F40401300E82273BEC0BF0CA
:1026A00031C182F40401300E82273BEC0BF032C1C1
:1026B00082F40401300E82273BEC0BF033C182F42C
:1026C0000401300E82273BEC0BF004012C0E826FCC
:1026D0003BEC0BF0200EF86EF76AF66A0401090075
:1026E000F5CF82F43BEC0BF00900F5CF82F43BEC24
:1026F0000BF00900F5CF82F43BEC0BF00900F5CFAD
:1027000082F43BEC0BF00900F5CF82F43BEC0BF0CC
:102710000900F5CF82F43BEC0BF00900F5CF82F411
:102720003BEC0BF00900F5CF82F43BEC0BF045ECF1
:102730000BF04EEF19F081B803D02FB0EBEF13F090
:102740008351630AD8A44CEF19F08451610AD8A4CC
:102750004CEF19F085516C0AD8A44CEF19F0865152
:10276000410A42E08651440A1BE08651420AD8B42D
:1027700007EF14F08651350AD8B4D8EF1AF0865115
:10278000360AD8B42DEF1BF08651370AD8B496EF2D
:102790001BF08651380AD8B4F4EF1BF04CEF19F057
:1027A0000798079A04017A0E826F3BEC0BF0040144
:1027B000780E826F3BEC0BF00401640E826F3BECF1
:1027C0000BF081A8EBEF13F00401550E826F3BEC88
:1027D0000BF0F0EF13F004014C0E826F3BEC0BF0AA
:1027E00045EC0BF04EEF19F00788079A04017A0EBA
:1027F000826F3BEC0BF00401410E826F3BEC0BF05F
:102800000401610E826F3BEC0BF0E1EF13F00798CF
:10281000078A04017A0E826F3BEC0BF00401420E32
:10282000826F3BEC0BF00401610E826F3BEC0BF00E
:10283000E1EF13F00101666725EF14F0676725EFFC
:1028400014F0686725EF14F0696715D04F6730EF13
:1028500014F0506730EF14F0516730EF14F0526706
:102860000AD00101000E006F000E016F000E026F12
:10287000000E036F120011B80AD00101620E046F3E
:10288000010E056F000E066F000E076F09D00101E3
:10289000A70E046F020E056F000E066F000E076F85
:1028A00066C100F167C101F168C102F169C103F1BC
:1028B0000CEC1FF003BFCDEF14F0119A119C010135
:1028C000000E046FA80E056F550E066F020E076FFF
:1028D00066C100F167C101F168C102F169C103F18C
:1028E00066C186F167C187F168C188F169C189F164
:1028F0000CEC1FF003BF0BD00101000E866FA80E79
:10290000876F550E886F020E896F118A119C0E0E0B
:102910002FEC09F0E8CF18F10F0E2FEC09F0E8CFFB
:1029200019F1100E2FEC09F0E8CF1AF1110E2FEC6F
:1029300009F0E8CF1BF155EC1EF086C104F187C108
:1029400005F188C106F189C107F10CEC1FF007827F
:1029500019EC1EF055EC1EF0079219EC1EF086C122
:1029600000F187C101F188C102F189C103F1079229
:1029700019EC1EF0CC0E046FE00E056F870E066F8B
:10298000050E076F0CEC1FF000C118F101C119F121
:1029900002C11AF103C11BF13BD0119C119A010134
:1029A000800E006F1A0E016F060E026F000E036F8D
:1029B0004FC104F150C105F151C106F152C107F1F7
:1029C0000CEC1FF003AF05D007EC20F0118C119A2E
:1029D00012000E0E2FEC09F0E8CF18F10F0E2FECBD
:1029E00009F0E8CF19F1100E2FEC09F0E8CF1AF139
:1029F000110E2FEC09F0E8CF1BF14FC100F150C1CF
:102A000001F151C102F152C103F1078219EC1EF02C
:102A100018C100F119C101F11AC102F11BC103F182
:102A200012000401730E826F3BEC0BF004012C0EBC
:102A3000826F3BEC0BF0078462C166F163C167F102
:102A400064C168F165C169F14BC14FF14CC150F1EE
:102A50004DC151F14EC152F157C159F158C15AF10E
:102A6000079437EC15F045EC0BF04EEF19F066C10A
:102A700000F167C101F168C102F169C103F101010F
:102A8000AAEC1FF06DEC1DF00401630E826F3BECAD
:102A90000BF004012C0E826F3BEC0BF04FC100F1E8
:102AA00050C101F151C102F152C103F10101AAEC7F
:102AB0001FF06DEC1DF00401660E826F3BEC0BF015
:102AC00004012C0E826F3BEC0BF007EC20F059C197
:102AD00000F15AC101F10101AAEC1FF06DEC1DF0EB
:102AE0000401740E826F3BEC0BF0120010820401A3
:102AF000530E826F3BEC0BF004012C0E826F3BEC0B
:102B00000BF083C32AF184C32BF185C32CF186C358
:102B10002DF187C32EF188C32FF189C330F18AC309
:102B200031F18BC332F18CC333F1010155EC20F04C
:102B3000CCEC1FF000C166F101C167F102C168F180
:102B400003C169F18EC32AF18FC32BF190C32CF11D
:102B500091C32DF192C32EF193C32FF194C330F1A1
:102B600095C331F196C332F197C333F1010155ECAE
:102B700020F0CCEC1FF000C14FF101C150F102C1B7
:102B800051F103C152F148EC20F099C32FF19AC3DF
:102B900030F19BC331F19CC332F19DC333F101018C
:102BA00055EC20F0CCEC1FF000C159F101C15AF1F5
:102BB00037EC15F004012C0E826F3BEC0BF0F0EFBC
:102BC00015F0118E19A002D019AE108C18BE02D0CB
:102BD00018A4108E8251520A02E10F8201D00F9286
:102BE0008251750A02E1108401D010948251550A75
:102BF00002E1108601D0109611A003D011A401D0DB
:102C00001084078410B25EEF16F010A44AEF16F09D
:102C1000B6C166F1B7C167F1B8C168F1B9C169F170
:102C2000BAC16AF1BBC16BF1BCC16CF1BDC16DF140
:102C3000BEC16EF1BFC16FF1C0C170F1C1C171F110
:102C4000C2C172F1C3C173F1C4C174F1C5C175F1E0
:102C5000C6C176F1C7C177F1C8C178F1C9C179F1B0
:102C6000CAC17AF1CBC17BF1CCC17CF1CDC17DF180
:102C7000CEC17EF1CFC17FF1D0C180F1D1C181F150
:102C8000D2C182F1D3C183F1D4C184F1D5C185F120
:102C900052EF16F062C166F163C167F164C168F179
:102CA00065C169F14BC14FF14CC150F14DC151F1BA
:102CB0004EC152F157C159F158C15AF107940FA0B2
:102CC00080EF16F0010192676DEF16F093676DEFDC
:102CD00016F094676DEF16F0956771EF16F080EFC0
:102CE00016F01AEC14F092C104F193C105F194C1ED
:102CF00006F195C107F10CEC1FF003BF14EF19F0BA
:102D00001AEC14F00101000E046F000E056F010EA5
:102D1000066F000E076F3DEC1FF011A02AD011A224
:102D200028D0AAEC1FF0296701D005D004012D0E90
:102D3000826F3BEC0BF030C182F40401300E82272D
:102D40003BEC0BF031C182F40401300E82273BECE6
:102D50000BF032C182F40401300E82273BEC0BF001
:102D600033C182F40401300E82273BEC0BF045ECBA
:102D70000BF012A8C3D012981AC01BF01B3A1B42CA
:102D8000070E1B1600011B50000AD8B44CEF17F0B9
:102D900000011B50010AD8B4D8EF16F000011B50F7
:102DA000020AD8B4D6EF16F07EEF17F07EEF17F0D8
:102DB00007EC20F02AC001F12BC000F1D8900133BC
:102DC0000033D890013300330101630E046F000E0D
:102DD000056F000E066F000E076F3DEC1FF0280E0A
:102DE000046F000E056F000E066F000E076F0CECEF
:102DF0001FF000C12DF007EC20F028C001F1019F69
:102E0000019D29C000F10101A40E046F000E056FA1
:102E1000000E066F000E076F3DEC1FF000C12CF096
:102E200000C104F101C105F102C106F103C107F1BE
:102E3000640E006F000E016F000E026F000E036F34
:102E40000CEC1FF0050E046F000E056F000E066FF0
:102E5000000E076F3DEC1FF000C104F101C105F148
:102E600002C106F103C107F107EC20F02DC000F10B
:102E70000CEC1FF000C12EF02EC0E8FF050F2D5CFA
:102E800003E78A847EEF17F02EC0E8FF0A0F2D5C5F
:102E900001E68A947EEF17F000C124F101C125F10B
:102EA00002C126F103C127F107EC20F00DEC20F060
:102EB0001A501F0BE8CF00F10101640E046F000EE1
:102EC000056F000E066F000E076F1DEC1FF024C18A
:102ED00004F125C105F126C106F127C107F10CEC6B
:102EE0001FF003BF02D08A9401D08A8424C100F16C
:102EF00025C101F126C102F127C103F100C124F16E
:102F000001C125F102C126F103C127F110AE4DD058
:102F1000109E00C108F101C109F102C10AF103C10B
:102F20000BF1AAEC1FF030C1D6F131C1D7F132C19B
:102F3000D8F133C1D9F108C100F109C101F10AC1C9
:102F400002F10BC103F101016C0E046F070E056F56
:102F5000000E066F000E076F0CEC1FF003BF04D0CD
:102F60000101550EDA6F1CD008C100F109C101F151
:102F70000AC102F10BC103F10101A40E046F060E98
:102F8000056F000E066F000E076F0CEC1FF003BFFD
:102F900004D001017F0EDA6F03D00101FF0EDA6F5A
:102FA0001C8E11AE14EF19F0119E24C100F125C141
:102FB00001F126C102F127C103F110A4E7EF17F0D8
:102FC0000401750E826F3BEC0BF0ECEF17F004017F
:102FD000720E826F3BEC0BF004012C0E826F3BEC07
:102FE0000BF0AAEC1FF02967FBEF17F00401200E8D
:102FF000826FFEEF17F004012D0E826F3BEC0BF099
:1030000030C182F40401300E82273BEC0BF031C159
:1030100082F40401300E82273BEC0BF004012E0EEB
:10302000826F3BEC0BF032C182F40401300E822738
:103030003BEC0BF033C182F40401300E82273BECF1
:103040000BF004016D0E826F3BEC0BF004012C0EB3
:10305000826F3BEC0BF04FC100F150C101F151C147
:1030600002F152C103F10101AAEC1FF06DEC1DF059
:103070000401480E826F3BEC0BF004017A0E826F64
:103080003BEC0BF004012C0E826F3BEC0BF066C1A5
:1030900000F167C101F168C102F169C103F10101E9
:1030A000AAEC1FF06DEC1DF00401630E826F3BEC87
:1030B0000BF004012C0E826F3BEC0BF066C100F1AB
:1030C00067C101F168C102F169C103F101010A0E92
:1030D000046F000E056F000E066F000E076F1DECEB
:1030E0001FF0000E046F120E056F000E066F000E2B
:1030F000076F3DEC1FF0AAEC1FF02AC182F4040117
:10310000300E82273BEC0BF02BC182F40401300E11
:1031100082273BEC0BF02CC182F40401300E822795
:103120003BEC0BF02DC182F40401300E82273BEC06
:103130000BF02EC182F40401300E82273BEC0BF021
:103140002FC182F40401300E82273BEC0BF030C11A
:1031500082F40401300E82273BEC0BF004012E0EAA
:10316000826F3BEC0BF031C182F40401300E8227F8
:103170003BEC0BF032C182F40401300E82273BECB1
:103180000BF033C182F40401300E82273BEC0BF0CC
:103190000401730E826F3BEC0BF004012C0E826F66
:1031A0003BEC0BF007EC20F059C100F15AC101F1E2
:1031B00078EC1AF00FB2E0EF18F00FA012EF19F050
:1031C00004012C0E826F3BEC0BF0200EF86EF76AB8
:1031D000F66A04010900F5CF82F43BEC0BF009001C
:1031E000F5CF82F43BEC0BF00900F5CF82F43BEC19
:1031F0000BF00900F5CF82F43BEC0BF00900F5CFA2
:1032000082F43BEC0BF00900F5CF82F43BEC0BF0C1
:103210000900F5CF82F43BEC0BF00900F5CF82F406
:103220003BEC0BF045EC0BF00F904EEF19F0040166
:10323000630E826F3BEC0BF004012C0E826F3BECB3
:103240000BF054EC19F004012C0E826F3BEC0BF0E8
:10325000C7EC19F004012C0E826F3BEC0BF043EC31
:103260001AF004012C0E826F3BEC0BF00101F80EFA
:10327000006FCD0E016F660E026F030E036F69ECD7
:1032800019F004012C0E826F3BEC0BF059EC1AF094
:1032900045EC0BF04EEF19F045EC0BF00301C26B5F
:1032A000079010925DEF1CF0D8900E0E2FEC09F0F5
:1032B000E8CF00F10F0E2FEC09F0E8CF01F1100E6E
:1032C0002FEC09F0E8CF02F1110E2FEC09F0E8CF56
:1032D00003F10101000E046F000E056F010E066F71
:1032E000000E076F3DEC1FF0AAEC1FF02AC182F41C
:1032F0000401300E82273BEC0BF02BC182F4040159
:10330000300E82273BEC0BF02CC182F40401300E0E
:1033100082273BEC0BF02DC182F40401300E822792
:103320003BEC0BF02EC182F40401300E82273BEC03
:103330000BF02FC182F40401300E82273BEC0BF01E
:1033400030C182F40401300E82273BEC0BF031C116
:1033500082F40401300E82273BEC0BF004012E0EA8
:10336000826F3BEC0BF032C182F40401300E8227F5
:103370003BEC0BF033C182F40401300E82273BECAE
:103380000BF004016D0E826F3BEC0BF01200120E7D
:103390002FEC09F0E8CF00F1130E2FEC09F0E8CF85
:1033A00001F1140E2FEC09F0E8CF02F1150E2FEC0D
:1033B00009F0E8CF03F101010A0E046F000E056F5A
:1033C000000E066F000E076F1DEC1FF0000E046F5D
:1033D000120E056F000E066F000E076F3DEC1FF01A
:1033E000AAEC1FF02AC182F40401300E82273BECC4
:1033F0000BF02BC182F40401300E82273BEC0BF062
:103400002CC182F40401300E82273BEC0BF02DC15D
:1034100082F40401300E82273BEC0BF02EC182F4C3
:103420000401300E82273BEC0BF02FC182F4040123
:10343000300E82273BEC0BF030C182F40401300ED9
:1034400082273BEC0BF004012E0E826F3BEC0BF05D
:1034500031C182F40401300E82273BEC0BF032C103
:1034600082F40401300E82273BEC0BF033C182F46E
:103470000401300E82273BEC0BF00401730E826FC7
:103480003BEC0BF012000A0E2FEC09F0E8CF00F134
:103490000B0E2FEC09F0E8CF01F10C0E2FEC09F028
:1034A000E8CF02F10D0E2FEC09F0E8CF03F178EF31
:1034B0001AF0060E2FEC09F0E8CF00F1070E2FEC02
:1034C00009F0E8CF01F1080E2FEC09F0E8CF02F186
:1034D000090E2FEC09F0E8CF03F178EF1AF00101A3
:1034E00007EC20F0078457C100F158C101F107949F
:1034F0000101E80E046F800E056F000E066F000ECE
:10350000076F1DEC1FF0000E046F040E056F000E18
:10351000066F000E076F3DEC1FF0880E046F130E50
:10352000056F000E066F000E076F0CEC1FF00A0E01
:10353000046F000E056F000E066F000E076F3DEC66
:103540001FF0AAEC1FF001012967ACEF1AF004018B
:10355000200E826FAFEF1AF004012D0E826F3BEC4C
:103560000BF030C182F40401300E82273BEC0BF0EB
:1035700031C182F40401300E82273BEC0BF032C1E2
:1035800082F40401300E82273BEC0BF004012E0E76
:10359000826F3BEC0BF033C182F40401300E8227C2
:1035A0003BEC0BF00401430E826F3BEC0BF012007E
:1035B00087C32AF188C32BF189C32CF18AC32DF16B
:1035C0008BC32EF18CC32FF18DC330F18EC331F13B
:1035D00090C332F191C333F10101296B55EC20F016
:1035E000CCEC1FF00101000E046F000E056F010E00
:1035F000066F000E076F1DEC1FF00E0E0C6E00C163
:103600000BF018EC09F00F0E0C6E01C10BF018EC6A
:1036100009F0100E0C6E02C10BF018EC09F0110E3F
:103620000C6E03C10BF018EC09F004017A0E826FE6
:103630003BEC0BF004012C0E826F3BEC0BF0040111
:10364000350E826F3BEC0BF004012C0E826F3BECCD
:103650000BF054EC19F0F0EF13F087C32AF188C394
:103660002BF189C32CF18AC32DF18BC32EF18CC3AE
:103670002FF18DC330F18EC331F190C332F191C37C
:1036800033F10101296B55EC20F0CCEC1FF0880ED2
:10369000046F130E056F000E066F000E076F11EC1E
:1036A0001FF0000E046F040E056F000E066F000E73
:1036B000076F1DEC1FF00101E80E046F800E056F0F
:1036C000000E066F000E076F3DEC1FF00A0E0C6E29
:1036D00000C10BF018EC09F00B0E0C6E01C10BF0E1
:1036E00018EC09F00C0E0C6E02C10BF018EC09F08E
:1036F0000D0E0C6E03C10BF018EC09F004017A0EEC
:10370000826F3BEC0BF004012C0E826F3BEC0BF054
:103710000401360E826F3BEC0BF004012C0E826F1D
:103720003BEC0BF043EC1AF0F0EF13F087C32AF1F7
:1037300088C32BF189C32CF18AC32DF18BC32EF1E1
:103740008CC32FF18DC330F18FC331F190C332F1AF
:1037500091C333F1010155EC20F0CCEC1FF0000EC9
:10376000046F120E056F000E066F000E076F1DEC42
:103770001FF001010A0E046F000E056F000E066FA8
:10378000000E076F3DEC1FF0120E0C6E00C10BF027
:1037900018EC09F0130E0C6E01C10BF018EC09F0D7
:1037A000140E0C6E02C10BF018EC09F0150E0C6E25
:1037B00003C10BF018EC09F004017A0E826F3BECA8
:1037C0000BF004012C0E826F3BEC0BF00401370E62
:1037D000826F3BEC0BF004012C0E826F3BEC0BF084
:1037E000C7EC19F0F0EF13F087C32AF188C32BF16F
:1037F00089C32CF18AC32DF18BC32EF18CC32FF119
:103800008DC330F18EC331F190C332F191C333F1E6
:103810000101296B55EC20F0CCEC1FF0880E046FF1
:10382000130E056F000E066F000E076F11EC1FF0F0
:10383000000E046F040E056F000E066F000E076F7A
:103840001DEC1FF00101E80E046F800E056F000EE5
:10385000066F000E076F3DEC1FF0060E0C6E00C1E8
:103860000BF018EC09F0070E0C6E01C10BF018EC10
:1038700009F0080E0C6E02C10BF018EC09F0090EED
:103880000C6E03C10BF018EC09F004017A0E826F84
:103890003BEC0BF004012C0E826F3BEC0BF00401AF
:1038A000380E826F3BEC0BF004012C0E826F3BEC68
:1038B0000BF059EC1AF0F0EF13F081B803D02FB0F1
:1038C0001BEF1DF007A8D5EF1CF00101800E006F63
:1038D0001A0E016F060E026F000E036F4BC104F14A
:1038E0004CC105F14DC106F14EC107F10CEC1FF0C2
:1038F00003BF1BEF1DF067EC1DF04BC100F14CC185
:1039000001F14DC102F14EC103F1078219EC1EF025
:1039100018C104F119C105F11AC106F11BC107F163
:10392000F80E006FCD0E016F660E026F030E036F6F
:103930000CEC1FF00E0E0C6E00C10BF018EC09F031
:103940000F0E0C6E01C10BF018EC09F0100E0C6E8E
:1039500002C10BF018EC09F0110E0C6E03C10BF054
:1039600018EC09F00784010107EC20F057C100F1C1
:1039700058C101F107940A0E0C6E00C10BF018EC4F
:1039800009F00B0E0C6E01C10BF018EC09F00C0ED7
:103990000C6E02C10BF018EC09F00D0E0C6E03C199
:1039A0000BF018EC09F01BEF1DF007AA1BEF1DF040
:1039B0000784010107EC20F057C100F158C101F163
:1039C0000794060E0C6E00C10BF018EC09F0070E00
:1039D0000C6E01C10BF018EC09F0080E0C6E02C160
:1039E0000BF018EC09F0090E0C6E03C10BF018EC8B
:1039F00009F0078462C100F163C101F164C102F101
:103A000065C103F10794120E0C6E00C10BF018ECA7
:103A100009F0130E0C6E01C10BF018EC09F0140E36
:103A20000C6E02C10BF018EC09F0150E0C6E03C100
:103A30000BF018EC09F00798079A040180518119DE
:103A40007F0B0DE09EA8FED714EE00F081517F0B96
:103A5000E126E750812B0F01AD6E1DEF1DF092EFB7
:103A60000AF018C100F119C101F11AC102F11BC11C
:103A700003F1000E046F000E056F010E066F000EBD
:103A8000076F3DEC1FF029A15CEF1DF02051D8B469
:103A90005CEF1DF018C100F119C101F11AC102F16A
:103AA0001BC103F1000E046F000E056F0A0E066FB6
:103AB000000E076F3DEC1FF01200010104510013CE
:103AC000055101130651021307510313120001019E
:103AD000186B196B1A6B1B6B12002AC182F404015C
:103AE000300E82273BEC0BF02BC182F40401300E28
:103AF00082273BEC0BF02CC182F40401300E8227AC
:103B00003BEC0BF02DC182F40401300E82273BEC1C
:103B10000BF02EC182F40401300E82273BEC0BF037
:103B20002FC182F40401300E82273BEC0BF030C130
:103B300082F40401300E82273BEC0BF031C182F499
:103B40000401300E82273BEC0BF032C182F40401F9
:103B5000300E82273BEC0BF033C182F40401300EAF
:103B600082273BEC0BF012002FC182F40401300ECF
:103B700082273BEC0BF030C182F40401300E822727
:103B80003BEC0BF031C182F40401300E82273BEC98
:103B90000BF032C182F40401300E82273BEC0BF0B3
:103BA00033C182F40401300E82273BEC0BF012008B
:103BB000060E1E6E060E1F6E060E206E1E2EDEEF09
:103BC0001DF01F2EDEEF1DF0202EDEEF1DF08B848A
:103BD000020E1E6E020E1F6E020E206E1E2EEEEFE5
:103BE0001DF01F2EEEEF1DF0202EEEEF1DF08B943A
:103BF0001200FF0E1F6E1FC020F0030E1E6E8B847E
:103C00001E2EFFEF1DF0030E1E6E202EFFEF1DF087
:103C10008B941FC020F0030E1E6E1E2E0DEF1EF0A3
:103C2000030E1E6E203E0DEF1EF01F2EFBEF1DF04B
:103C300012000101005305E1015303E1025301E1C8
:103C4000002BDCEC1EF007EC20F03951006F3A51EC
:103C5000016F420E046F4B0E056F000E066F000ED3
:103C6000076F1DEC1FF000C104F101C105F102C195
:103C700006F103C107F118C100F119C101F11AC120
:103C800002F11BC103F107B24AEF1EF011EC1FF065
:103C90004CEF1EF00CEC1FF000C118F101C119F13E
:103CA00002C11AF103C11BF1120007EC20F059C147
:103CB00000F15AC101F1060E2FEC09F0E8CF04F132
:103CC000070E2FEC09F0E8CF05F1080E2FEC09F0F4
:103CD000E8CF06F1090E2FEC09F0E8CF07F10CEC64
:103CE0001FF000C124F101C125F102C126F103C179
:103CF00027F1290E046F000E056F000E066F000EEF
:103D0000076F1DEC1FF0EE0E046F430E056F000EE3
:103D1000066F000E076F11EC1FF024C104F125C1DE
:103D200005F126C106F127C107F11DEC1FF000C106
:103D30001CF101C11DF102C11EF103C11FF1120EE0
:103D40002FEC09F0E8CF04F1130E2FEC09F0E8CFC7
:103D500005F1140E2FEC09F0E8CF06F1150E2FEC4B
:103D600009F0E8CF07F10D0E006F000E016F000E95
:103D7000026F000E036F1DEC1FF0180E046F000E93
:103D8000056F000E066F000E076F3DEC1FF01CC1A3
:103D900004F11DC105F11EC106F11FC107F111ECAF
:103DA0001FF06A0E046F2A0E056F000E066F000EDC
:103DB000076F0CEC1FF01200BF0EFA6E200E3A6F68
:103DC000396BD8900037013702370337D8B0EDEFA1
:103DD0001EF03A2FE2EF1EF039073A070353D8B42A
:103DE00012000331070B80093F6F03390F0B010FDE
:103DF000396F80EC5FF0406F390580EC5FF0405D1B
:103E0000405F396B3F33D8B0392739333FA902EFD0
:103E10001FF040513927120001012CEC20F0D8B0DE
:103E20001200010103510719346FEFEC1FF0D89015
:103E30000751031934AF800F12000101346B13ECEA
:103E400020F0D8A029EC20F0D8B01200FEEC1FF032
:103E500007EC20F01F0E366F3FEC20F00B35D8B08A
:103E6000EFEC1FF0D8A00335D8B01200362F2CEF9E
:103E70001FF034B116EC20F012000101346B045134
:103E80000511061107110008D8A013EC20F0D8A0E6
:103E900029EC20F0D8B01200086B096B0A6B0B6B91
:103EA0003FEC20F01F0E366F3FEC20F007510B5D0A
:103EB000D8A467EF1FF006510A5DD8A467EF1FF082
:103EC0000551095DD8A467EF1FF00451085DD8A023
:103ED0007AEF1FF00451085F0551D8A0053D095F36
:103EE0000651D8A0063D0A5F0751D8A0073D0B5FD9
:103EF000D8900081362F54EF1FF034B116EC20F02B
:103F0000346B13EC20F0D89043EC20F007510B5D9C
:103F1000D8A497EF1FF006510A5DD8A497EF1FF0C1
:103F20000551095DD8A497EF1FF00451085DD8A092
:103F3000A6EF1FF0003FA6EF1FF0013FA6EF1FF016
:103F4000023FA6EF1FF0032BD8B4120034B116ECD9
:103F500020F012000101346B13EC20F0D8B01200F5
:103F600048EC20F0200E366F003701370237033758
:103F700011EE33F00A0E376FE7360A0EE75CD8B061
:103F8000E76EE552372FBCEF1FF0362FB4EF1FF06E
:103F900034B12981D890120001010A0E346F200E2D
:103FA000366F11EE29F03451376F0A0ED890E65271
:103FB000D8B0E726E732372FD7EF1FF003330233AD
:103FC00001330033362FD1EF1FF0E750FF0FD8A099
:103FD0000335D8B0120029B116EC20F012000451BC
:103FE00000270551D8B0053D01270651D8B0063D40
:103FF00002270751D8B0073D032712000051086F70
:104000000151096F02510A6F03510B6F1200010138
:10401000006B016B026B036B12000101046B056BFB
:10402000066B076B12000335D8A012000351800BFA
:10403000001F011F021F031F003F26EF20F0013F5A
:1040400026EF20F0023F26EF20F0032B342B032530
:1040500012000735D8A012000751800B041F051F5E
:10406000061F071F043F3CEF20F0053F3CEF20F008
:10407000063F3CEF20F0072B342B072512000037BA
:10408000013702370337083709370A370B37120071
:104090000101296B2A6B2B6B2C6B2D6B2E6B2F6BFD
:1040A000306B316B326B336B120001012A510F0BF5
:1040B0002A6F2B510F0B2B6F2C510F0B2C6F2D5187
:1040C0000F0B2D6F2E510F0B2E6F2F510F0B2F6FCC
:1040D00030510F0B306F31510F0B316F32510F0BCD
:1040E000326F33510F0B336F120000011650FF0A6D
:1040F00001E11200390EC86E800EC76E280EC66E22
:10410000000EC56E1550000AD8B4B0EF20F015505F
:10411000010AD8B4C9EF20F01550020AD8B4E2EF72
:1041200020F01550030AD8B4FBEF20F01550040A14
:10413000D8B423EF21F01550050AD8B43CEF21F094
:104140001550060AD8B455EF21F01550070AD8B417
:104150006EEF21F01550080AD8B487EF21F0120055
:104160001650000AD8B4A6EF21F01650010AD8B4B0
:10417000AAEF21F01650020AD8B4AEEF21F0165083
:10418000030AD8B4B2EF21F01650040AD8B425EFD0
:1041900022F01650000AD8B4BAEF21F01650010AE6
:1041A000D8B4BEEF21F01650020AD8B4C2EF21F005
:1041B0001650030AD8B4C6EF21F01650040AD8B43A
:1041C00025EF22F01650000AD8B4CAEF21F016509D
:1041D000010AD8B4CEEF21F01650020AD8B4D2EFBB
:1041E00021F01650030AD8B4D6EF21F01650040A75
:1041F000D8B425EF22F01650000AD8B4E3EF21F02E
:104200001650010AD8B4E7EF21F01650020AD8B4CC
:10421000EBEF21F01650030AD8B4FFEF21F016504F
:10422000040AD8B403EF22F01650050AD8B407EFF9
:1042300022F01650060AD8B40BEF22F01650070AE7
:10424000D8B40EEF22F01650000AD8B412EF22F0C4
:104250001650010AD8B416EF22F01650020AD8B44C
:104260001AEF22F01650030AD8B41EEF22F01650AF
:10427000040AD8B421EF22F01650000AD8B429EF6E
:1042800022F01650010AD8B42DEF22F01650020A7F
:10429000D8B431EF22F01650030AD8B435EF22F02B
:1042A0001650040AD8B425EF22F01650000AD8B4EC
:1042B0003FEF22F01650010AD8B443EF22F0165017
:1042C000020AD8B447EF22F01650030AD8B44BEFD5
:1042D00022F01650040AD8B425EF22F01650000A36
:1042E000D8B44CEF22F01650010AD8B450EF22F0A7
:1042F0001650020AD8B454EF22F01650030AD8B46C
:1043000058EF22F01650040AD8B425EF22F01650C8
:10431000000AD8B459EF22F01650010AD8B45DEF64
:1043200022F01650020AD8B461EF22F01650030AA8
:10433000D8B465EF22F01650040AD8B466EF22F024
:104340001650050AD8B469EF22F012009E96C58077
:10435000162A1200E20EC96E162A1200770EC96ED6
:10436000162A1200020EE86E8AB4E88AE8CFC9FF66
:10437000162A12009E96C580162A1200E20EC96EF9
:10438000162A1200790EC96E162A1200000EC96E86
:10439000162A12009E96C580162A1200E20EC96ED9
:1043A000162A12007A0EC96E162A120018BC03D003
:1043B000DAC1E8FF04D01850E844E8441F09E8CF08
:1043C000C9FF162A12009E96C580162A1200E20E18
:1043D000C96E162A120011BA03D011BC01D003D045
:1043E000050E156E3ED00101D667FBEF21F0100ED1
:1043F000C96EFDEF21F0D6C1C9FF162A1200D7C140
:10440000C9FF162A1200D8C1C9FF162A1200D9C145
:10441000C9FF162A1200C584162A1200FF0E166E56
:104420001D9E12009E96C580162A1200E20EC96ECD
:10443000162A1200760EC96E162A1200C584162A94
:104440001200FF0E166E1D9E1200C584152A166AF4
:1044500012009E96C580162A1200E20EC96E162A18
:1044600012007B0EC96E162A120011AA04D0230E68
:10447000C96E162A12001C0EC96E162A12009E96CC
:10448000C580162A1200E20EC96E162A12007C0E92
:10449000C96E162A1200E9D79E96C580162A120008
:1044A000E20EC96E162A12007D0EC96E162A12007F
:1044B000DCD79E96C580162A1200E20EC96E162A17
:1044C00012007E0EC96E162A1200CFD7C584162A96
:1044D0001200FF0E166E1D9E12001650FF0AD8B471
:1044E0002BEF23F0390EC86E800EC76E280EC66EF5
:1044F000000EC56E1550000AD8B486EF22F0155094
:10450000010AD8B49AEF22F02BEF23F01650000ADC
:10451000D8B4D8EF22F01650010AD8B4DCEF22F05C
:104520001650020AD8B4E6EF22F01650030AD8B4A7
:10453000E9EF22F01650000AD8B4EFEF22F016503F
:10454000010AD8B4F3EF22F01650020AD8B4FDEFF6
:1045500022F01650030AD8B400EF23F01650040AD4
:10456000D8B406EF23F01650050AD8B409EF23F0AB
:104570001650060AD8B40FEF23F01650070AD8B425
:1045800012EF23F01650080AD8B418EF23F0165093
:10459000090AD8B41BEF23F016500A0AD8B421EF49
:1045A00023F016500B0AD8B424EF23F02BEF23F09E
:1045B0009E96C5802AEF23F017B004D04E0EC96E28
:1045C0002AEF23F0500EC96E2AEF23F0C5842AEF9C
:1045D00023F0152AFF0E166E12802BEF23F09E9605
:1045E000C5802AEF23F017B004D04F0EC96E2AEF12
:1045F00023F0510EC96E2AEF23F0C5862AEF23F06F
:10460000C9CF24F0C59AC5882AEF23F0C5862AEFC2
:1046100023F0C9CF25F0C59AC5882AEF23F0C586B7
:104620002AEF23F0C9CF26F0C59AC5882AEF23F0D8
:10463000C5862AEF23F0C9CF27F0C58AC5882AEF9F
:1046400023F0C5842AEF23F0FF0E166E12861D9C00
:104650002BEF23F0162A120012B012D012B213D090
:1046600012B414D012A6120007B01200129624C081
:1046700028F025C029F026C02AF027C02BF0120010
:10468000129012821200129212841200000116502F
:0E469000FF0A04E11294166A6DEC22F012008B
:10BF0000E844F926000C160C2B0C3F0C520C640C68
:10BF1000760C860C960CA50CB30CC10CCF0CDC0C6B
:06BF2000E80CF40C000C1B
:00000001FF
